:1000000001308A0071290000D3346D38EC32202A87
:10001000E832F236EF36653AE8327210A0060A008E
:10002000D63C73366532EE3220265321A0126C2C5A
:10003000A0060A0083168611831286110830F80084
:1000400021280000F8173228F813B00C0318861581
:10005000031C8611781732287813F80B25283028CE
:10006000000086153F308400840B34280000F81B04
:100070002428781B2C280800831603178C170C14CF
:100080000000000083120C087F3903198028031335
:10009000AC0003170D080313AD0003170F0803137B
:1000A000AE002C08B0001A202D0803178D00031392
:1000B0002E0803178F0083168C170C140000000005
:1000C00083120C0D0E0D7F39031980280313AC0029
:1000D00003170D080313AD0003170F080313AE0039
:1000E0002C08B0001A202D0803178D0003132E08CA
:1000F00003178F008D0A03198F0A03133C28031777
:1001000003138A110A12D9290830F800000086105A
:100110008316861000008312AC0D0610031C932872
:100120008316061483120318982883160610831268
:10013000831686148312861C9B28F80B86280000E1
:100140008610831686100000061400000000861436
:100150008312861CA928F80100000618781486105E
:100160008316861083120610831606108312080069
:100170002C308400831300080319CB280230F800C8
:10018000F701F70BC128F80BC0289730F700F70BE1
:10019000C728800BBE2808000830AD007708AE00E5
:1001A00083160614000086148312861CD5280618B0
:1001B0000314061C0310F80D00008316861083122A
:1001C0008610AD0BD028831606140000831206108B
:1001D0002E080319EE2883160610831200008316DA
:1001E00086148312861CF22800008610831686105F
:1001F0000000831206108316061083120800AD1B40
:1002000011290F30F7002C0EF7050A30770203187A
:100210000C293030F7070E292D08F7077708B000B2
:100220001A200F30AC050A302C020318192930307F
:100230001B29AD132D08AC072C08B0001A200800AC
:10024000831603178C170C140000000003184F29A5
:1002500083120C087F390313AD0003170D08031335
:10026000AE0003170F080313AF002D08B0001A20CB
:100270002E0803178D0003132F0803178F00831612
:100280008C170C140000000083120313AC0B4929D7
:100290004C29831603174F296E29831603178312DF
:1002A0000C0D0E0D7F390313AD0003170D0803135A
:1002B000AE0003170F080313AF002D08B0001A207B
:1002C0002E0803178D0003132F0803178F008D0AC4
:1002D00003198F0A03100313AC0B20298A110A1289
:1002E000452B840183131F308305713083168F00E3
:1002F0000F08861183128615831603170908C03963
:10030000890003131F129F12003003178800831205
:10031000870188018901FF300313A00083160317AA
:100320000908C039890003131F129F1200300317F8
:100330008800831203131F139F1383169F138312C6
:100340001F149412A012200883168700831220160F
:100350002008831687008312A011200883168700C7
:100360000130831294000030831694000108C739CD
:1003700008388100831290010030F80092000030AC
:10038000831692008312201520088316870083129B
:10039000970183169B019C0101309D008312031776
:1003A00087018801890104308D0000308F0003131C
:1003B0003C28A701A901831606140000861400003A
:1003C000831206108316061000008312861083160F
:1003D0008610AA308312AC0084206130AC008420E7
:1003E000831606140000861400008312861CF6296A
:1003F00006108316061000008312861083168610DE
:10040000AA308312AC008420AC018420831606102D
:10041000000086148312861C0B2A00000F2A00009D
:1004200083160614000001308312AC00B820831636
:1004300006140000861400008312061083160610AE
:1004400000008312861083168610AA308312AC0037
:1004500084203E30AC0084208316061400008614ED
:1004600000008312861C322A061083160610000034
:100470008312861083168610AA308312AC00842063
:100480005030AC00842083160610000086148312BE
:10049000861C482A00004C2A00008316061400001F
:1004A00001308312AC00B8208316061400008614B5
:1004B00000008312061083160610000083128610B7
:1004C00083168610AA308312AC0084203F30AC0023
:1004D0008420831606140000861400008312861CF4
:1004E0006F2A0610831606100000831286108316EA
:1004F0008610AA308312AC0084200230AC00842025
:1005000083160610000086148312861C852A0000BC
:10051000892A000083160614000001308312AC0003
:10052000B8208316061400008614000083120610FB
:100530008316061000008312861083168610AA30D8
:100540008312AC0084204530AC008420831606144E
:100550000000861400008312861CAC2A0610831645
:10056000061000008312861083168610AB308312AB
:10057000AC008420F701CC207808AA00831606106E
:10058000000086148312861CC32A0000C72A0000BC
:10059000831606140000061400008614000083125F
:1005A000061083160610000083128610831686102C
:1005B000AA308312AC0084204630AC00842083161D
:1005C00006140000861400008312861CE52A06101B
:1005D0008316061000008312861083168610AB3037
:1005E0008312AC008420F701CC207808AB0083167E
:1005F0000610000086148312861CFC2A0000002BC3
:10060000000083160614000001308312AC00B820ED
:100610005630B0001A204C30B0001A202030B00004
:100620001A202B08AC003730AD00FF202030B0007E
:100630001A200D30B0001A200A30B0001A204C30B9
:10064000B0001A204830B0001A202030B0001A2024
:100650002A08AC003730AD00FF202030B0001A204F
:100660000D30B0001A200A30B0001A20AA08031D6D
:10067000552B0130A702103003178D0000308F007A
:1006800003100D300313AC0020292708AC003730CD
:10069000AD00FF202030B0001A200D30B0001A202D
:1006A0000A30B0001A20532B8E2B8316061400003C
:1006B00086140000831206108316061000008312B1
:1006C000861083168610AA308312AC008420453031
:1006D000AC008420831606140000861400008312E8
:1006E000861C702B061083160610000083128610DD
:1006F00083168610AA308312AC008420AC018420BB
:1007000083160610000086148312861C852B0000B9
:10071000892B00008316061400008312831606142A
:1007200000008614000083120610831606100000D5
:100730008312861083168610AA308312AC008420A0
:100740006030AC008420831606140000861400007C
:100750008312861CA92B0610831606100000831234
:10076000861083168610AA308312AC0084202708D6
:10077000AC00842083160610000086148312861CA9
:10078000BF2B0000C32B00008316061400000130AD
:0E0790008312A7076430AC00B820DB29630099
:04400E00F52CFF3F4F
:00000001FF
